:020000040000FA
:0200000075D1B8
:08000800F2B20CD0F2B40CD0EE
:020010001100DD
:080018000B6ED8CF0AF0E0CF17
:1000200009F03AD0F2921100F2940F0E8912921256
:10003000EC0E8A1293120C50F92620D00FD089961C
:100040000F0E0D140809921AE00E0D14931A0DB636
:100050009396938410B693940C6A1DD089940F0ED6
:100060000E140409921AE00E0E14931A0EB493960D
:1000700093842BA29394040E0C6E0DD089900F0ED6
:100080000F140109921AE00E0F14931A0FB09396F1
:10009000020E0C6E00D011009E921B661B061D2ED8
:1000A0000FD0640E1D6E202A1E2E04D03C0E1E6E34
:1000B0001C661C061F2E04D03C0E1F6E1AAE212A91
:1000C000172E0AD0020E176E1850500B196E805062
:1000D000500B186E1962188E09C0E0FF0B500AC051
:0400E000D8FF100035
:100200006F6F6F066FAB6F8F6FC66FCD6FED6F0740
:100210006FEF6FCF066F060606AB068F06C606CDDC
:1002200006ED060706EF06CFAB6FAB06ABABAB8FA9
:10023000ABC6ABCDABEDAB07ABEFABCF8F6F8F06E4
:100240008FAB8F8F8FC68FCD8FED8F078FEF8FCFB7
:10025000C66FC606C6ABC68FC6C6C6CDC6EDC60738
:10026000C6EFC6CFCD6FCD06CDABCD8FCDC6CDCD34
:10027000CDEDCD07CDEFCDCFED6FED06EDABED8F35
:10028000EDC6EDCDEDEDED07EDEFEDCF076F070618
:1002900007AB078F07C607CD07ED070707EF07CFA7
:1002A000EF6FEF06EFABEF8FEFC6EFCDEFEDEF07A0
:1002B000EFEFEFCFCF6FCF06CFABCF8FCFC6CFCD86
:1002C000CFEDCF07CFEFCFCF00010102020304042F
:1002D00005060607080809090000000200040005D9
:1002E000000700090101010301040106D350700950
:1002F000D36E896A7F0EC16E500E926E8A6A030EAB
:10030000936EFDEC01F011EC02F00850AA0A0AE02D
:10031000FDEC01F0230E046E0A0E056E010E026E56
:10032000140E066E500E186E050E176E050E406EFA
:10033000C30ED56ED66ACA6ACC6A2B0ECA6ED00EB0
:10034000CB6ECA84F26A9D6AA06A9E6AC00EF06E85
:10035000C50EF16E9F6AD08E9D82E00EF26EEF0E9A
:100360000F6EEF0E0E6EEF0E0D6E898E8A88FA0EEE
:10037000F9EC01F0899E8A98B7EC02F0FDE140ECBF
:1003800002F0CC0E96EC02F0440E96EC02F02C0E2D
:100390000F6E6F0E0E6ECD0E0D6EC80EF9EC01F0E5
:1003A000ADEC06F018A8DCEC04F018ACFDEC06F09F
:1003B00066EC03F09AEC04F0BEEC04F0C7EC04F039
:1003C000F1D7116E112611C0F6FF020EF76E09006B
:1003D000F5CF11F00800F5CF12F01200189E1B6E39
:1003E000189018AE03D0189E188012001B66F9D71B
:1003F00012001B6E1B66FED7120000EE00F0EE6AC4
:10040000EAA0FDD71200AA0E086E426A090E436EDA
:1004100000EE00F0EE501EEC02F0422A432EFAD716
:100420001200426A090E436E00EE00F042502FECBB
:1004300002F0EE6E422A432EF9D71200A6B2FED782
:10044000A86E42C0A9FFA69EA69CA684F29E550E49
:10045000A76EAA0EA76EA682F28EA6941200A96EAF
:10046000A69EA69CA680A8501200000000000000D6
:100470000000000000000000252EF7D70000120049
:100480000000938000000000000000000000000059
:1004900081909390770E256E000000000000000010
:1004A00035EC02F0F29E93800D0E256E00000000E8
:1004B0000000000035EC02F08150F28E010B266E38
:1004C0004F0E256E000000000000000035EC02F029
:1004D0001200080E246EF29E81909390000000009E
:1004E000000000000000000000000000000000000C
:1004F00093800000000000000000000000000000E9
:100500000000000000008150010BFF0F27320000A7
:100510000000090E256E000000000000000035EC10
:1005200002F0F28E242ED7D727501200276E080E25
:10053000246EF29E81909390010E256E00000000C3
:100540000000000035EC02F02732D8B093800B0E8B
:10055000256E000000000000000035EC02F09380E2
:10056000000000000000F28E242EE3D712000000ED
:10057000938000000000000000000000000081A047
:100580004ED040EC02F040EC02F026500EE1330E6B
:1005900096EC02F069EC02F02A6E100E2A1804E0C4
:1005A000280E2A1801E09DD1000C93800000000065
:1005B000000000000000000081A031D081909390E5
:1005C000770E256E000000000000000035EC02F000
:1005D000F29E93800C0E416E010E256E000000000D
:1005E0000000000035EC02F081A030D0412EF4D79D
:1005F000F28E2B828A98898EE10E0F6E680E0E6E37
:10060000E00E0D6EC80EF9EC01F0670E0F6EAC0E29
:100610000E6EE00E0D6EC80EF9EC01F0EAD7F28E08
:100620002B828A98898EE10E0F6E680E0E6EE00E98
:100630000D6EC80EF9EC01F0ADEC06F0680E0E6E12
:10064000AC0E0D6EC80EF9EC01F0E9D7F28E2B82DC
:100650008A98898EE10E0F6E680E0E6EE00E0D6E9A
:10066000C80EF9EC01F0A00E0F6EE90E0E6ECD0E65
:100670000D6EC80EF9EC01F0E9D7F28E2B82690EEF
:100680000F6EA00E0E6E690E0D6EC80EF9EC01F025
:10069000E90E0F6EA00E0E6EA00E0D6EC80EF9ECD8
:1006A00001F0010CF28E2B82A00E0F6EAE0E0E6EBC
:1006B0000D6AC80EF9EC01F0E90E0F6EA00E0E6E79
:1006C000A00E0D6EC80EF9EC01F0010C69EC02F001
:1006D000010F0AE00A0EF9EC01F0342A140E34621C
:1006E000010C346A52EF03F0346A40EC02F02666E3
:1006F000D5EF02F0CC0E96EC02F0BE0E96EC02F0B6
:1007000069EC02F0286E316A326A87EC04F069EC19
:1007100002F0296E87EC04F069EC02F087EC04F03B
:1007200069EC02F087EC04F069EC02F087EC04F06D
:1007300069EC02F087EC04F069EC02F02D6E87ECB6
:1007400004F069EC02F02C6E87EC04F069EC02F026
:1007500087EC04F0315091E132A08FE040EC02F0E0
:10076000CC0E96EC02F0440E96EC02F04066404E41
:1007700002D01A8409D028503A5C2950D8A0010F21
:100780003B5C800BD8A406D028C03AF029C03BF0CF
:100790002DC03EF01AB409D028503C5C2950D8A096
:1007A000010F3D5C800BD8B407D028C03CF029C0B5
:1007B0003DF02DC03FF01A942B6A2950F00BF00A3F
:1007C000D8B42B80100E2A1804E0280E2A1825E031
:1007D00088D0D89028302E6E100E2C180AE028B041
:1007E00005D02F6A2BA024D02E0622D0050E2F6E06
:1007F0001FD02D502C5E2BA006D02C5002E12E06CF
:1008000002D010082C6E020EF76E2CC0F6FFC80E38
:10081000F6260800F5502F6E0BD00F0E28142C6E04
:10082000070E29142E6EF00E28142E122E3AE3D73E
:100830002BA003D02E507F082E6E2EC038F02FC074
:1008400039F007A006D0B2EC06F036C038F037C059
:1008500039F0C70E38640CD0C80E385CE1EC01F0FA
:1008600011C00EF012C00DF0AB0E0F6E2B82000CFB
:10087000630E38640CD0640E385CE1EC01F011C0FA
:100880000EF012C00DF0060E0F6E2B82000C3850C9
:10089000E1EC01F054EC04F02BB2000C3950E1EC27
:1008A00001F012C00DF0000C2BA004D007A00BD05B
:1008B0002BB409D06F0E116201D0116A11C00FF074
:1008C00012C00EF01200800E0F6E0A0E386003D0B8
:1008D00012C00EF0120011C00EF012C00DF02B82EB
:1008E0001200F28E2B828A98898E200E0F6EAE0E29
:1008F0000E6E0D6AC80EF9EC01F0E90E0F6EA00E37
:100900000E6EA00E0D6EC80EF9EC01F0EAD7306E37
:10091000080E336E30503118136E1330315001E32E
:10092000180A136E1330316E01E032803042332EDC
:10093000F1D7120000B00BD02BB018D0385006649D
:1009400001D014D00250062438600AD016D02BB043
:1009500003D0385006640AD00250065C38600DD0CF
:100960001C660BD0819801C01CF007D01C6605D016
:100970001ABE03D0818801C01CF0120038500464F4
:1009800004D0056002D0809E1200808E12000366A3
:1009900001D002D081B206D010961A9E3C0E1F6E76
:1009A000216A120010860350216001D012001DB48C
:1009B00010961A8E819812001A822B82206A020EDB
:1009C000206061D0ADEC06F018A8F9D7280E226E91
:1009D000030E236E06506BEC06F018AC01EC05F02C
:1009E0000F0E18B0F9EC01F0189018A822EC05F0E1
:1009F0000F0E18B0F9EC01F01890050E2064E6D740
:100A00005ED1206A18BC12002250EEEC01F0232EB9
:100A10000AD0030E236E22060A0E226004D00A0EAC
:100A2000226E18B01200062A640E07B0D40E0664B7
:100A300004D0640E07B0D40E066E06506BEC06F0C0
:100A40001A80DFD7206A18B812002250EEEC01F0AD
:100A5000232E0AD0030E236E22060A0E226004D033
:100A60000A0E226E18B012000606010E07B0200E04
:100A7000066004D0010E07B0200E066E06506BEC27
:100A800006F01A80DFD71A822B82CD0E0F6EE90E88
:100A90000E6EE00E0D6E6E0E68EC06F0690E0F6EB7
:100AA000800E0E6EE60E0D6EC80EEEEC01F0ADEC93
:100AB00006F0E60E00B0690E0D6E95EC06F018A873
:100AC0000CD018BCFAD7002A020E0060006AE60EAD
:100AD00000B0690E0D6E1A80F0D768EC06F0AE0E0D
:100AE0000F6E680E0E6ECE0E0D6EC80EEEEC01F09F
:100AF000ADEC06F001506BEC06F095EC06F018A892
:100B00000BD018BCFAD7012A100E0160016A0150FF
:100B10006BEC06F01A80F1D768EC06F0E60E0F6E6B
:100B2000CE0E0E6ECD0E0D6EC80EEEEC01F0ADECDD
:100B300006F002506BEC06F095EC06F018A80BD00E
:100B400018BCFAD7022A090E0260026A02506BEC46
:100B500006F01A80F1D768EC06F0AC0E0F6EAE0E00
:100B60000E6EAC0E0D6EC80EEEEC01F0ADEC06F0A4
:100B700003506BEC06F095EC06F018A80BD018BCEF
:100B8000FAD7032A0B0E0360036A03506BEC06F0DE
:100B90001A80F1D768EC06F0E60E0F6E200E0E6E8E
:100BA000E70E0D6EC80EEEEC01F0ADEC06F0045051
:100BB0006BEC06F095EC06F0280E226E030E236E09
:100BC00018A822D018BCF6D718BCF6D72250EEECE5
:100BD00001F0232E0AD0030E236E22060A0E226095
:100BE00004D00A0E226E18B0E7D7042A640E07B0AC
:100BF000D40E046404D00A0E07B0320E046E045002
:100C00006BEC06F01A80DCD768EC06F0680E0F6E0D
:100C1000AC0E0E6EE70E0D6EC80EEEEC01F0ADECF4
:100C200006F005506BEC06F095EC06F0280E226EEF
:100C3000030E236E18A822D018BCF6D718BCF6D71E
:100C40002250EEEC01F0232E0AD0030E236E220672
:100C50000A0E226004D00A0E226E18B0E7D7052AC9
:100C6000640E07B0D40E056404D0000E07B0200E49
:100C7000056E05506BEC06F01A80DCD768EC06F0C8
:100C8000690E0F6E800E0E6EE10E0D6EC80EEEEC4C
:100C900001F0ADEC06F0690E07B0E10E0D6E95ECBB
:100CA00006F018A80CD018BCFAD7072A020E076065
:100CB000076A690E07B0E10E0D6E1A80F0D768EC76
:100CC00006F01A922B921AB003EC02F01A9012005E
:100CD00018A8FED71200146EC70E14640BD0C80EED
:100CE000145CE1EC01F011C00EF012C00DF0AB0E7F
:100CF0000F6E1200630E14640BD0640E145CE1ECF2
:100D000001F011C00EF012C00DF0060E0F6E1200B1
:100D10000F6A1450E1EC01F06F0E116201D0116AFC
:100D200011C00EF012C00DF012000FC014F00EC072
:100D300015F00DC016F00F6A0E6A0D6A0A0EEEEC81
:100D400001F014C00FF015C00EF016C00DF018B071
:100D50001200140EEEEC01F012000F6A0E6A0D6A1A
:100D60002B821200090E2E02E7EC06F0F3CF36F0CC
:100D7000F450F424376E2F502F24F66E020EF76EC7
:100D8000D80EF6260900F55036260800F55037240F
:100D90000700356E0F0B376E35380F0B36262BB02C
:100DA00007D02B942B9E200E3626D8B02B8E120007
:100DB00036502008366E04E700082B84366E06D0C5
:100DC0002B94375003E00A08376E36061200080EDF
:100DD000356E050EF0EC06F0352EFCD7F33612001A
:100DE000F336F436D8A003D0F45ED8801200F45E57
:100DF000D8B01200F426D8901200206A040E2060A9
:100E00003BD02B82E60E0F6E200E0E6E0D6A18ACD4
:100E1000F5D7640EF9EC01F0ADEC06F02B923DC075
:100E200029F03CC028F03FC02DF0DCEC03F0B40EFC
:100E3000F9EC01F0ADEC06F0320EF9EC01F02B828A
:100E4000680E0F6EAC0E0E6E0D6A640EF9EC01F0BA
:100E5000ADEC06F02B923BC029F03AC028F03EC022
:100E60002DF0DCEC03F0B40EF9EC01F0ADEC06F083
:100E7000320EF9EC01F01200020E406E2B82690E68
:100E80000F6E680E0E6EA00E0D6EB40EF9EC01F032
:020E900012004E
:020000040030CA
:03000100080A1ECC
:020005008081F8
:0600080003C003E0034009
:00000001FF
